:101C000011241FBECFE5D4E0DEBFCDBF10E0A0E6BB
:101C1000B0E0EAE2FFE102C005900D92A036B10704
:101C2000D9F710E0A0E6B0E001C01D92A23AB107DA
:101C3000E1F714C000C008955D9BFECF8CB90895F4
:101C40005F9BFECF8CB1992708958DE4F5DF8BE47F
:101C5000F3DF82E4F1DF8CE4EFDF0895CFE5D4E039
:101C6000DEBFCDBFE0E0F0E004917F01992490BC9D
:101C700080E189B9599A88E18AB986E880BDEF0187
:101C8000192D5F9B0BC0113029F48CB18A3A49F1B0
:101C900010E004C08CB18B3109F411E0CE01219623
:101CA00084369105C8F00F3F41F0002331F0E091F8
:101CB0006000F091610009950FC08AE0BDDF8DE002
:101CC000BBDF86E5B9DF80E3B7DF8EE2B5DF81E316
:101CD000B3DF8AE3B1DF05C080E29EE40197F1F74C
:101CE000D0CFB3DFADDF813611F489E51CC181347B
:101CF00061F4A6DFE82EFF24FE2CEE24A1DF992755
:101D0000E82AF92AF694E794E1C0823631F489E5AD
:101D100093DF80E091DF80E406C1823409F070C077
:101D20008FDF8EDFD82E8CDF082FB2E6AB2EB0E02F
:101D3000BB2E10E0E5010894A11CB11C1D1510F488
:101D40007FDF01C08FEF88831F5F103498F336E781
:101D5000931609F0C9C0063409F03CC08FEFE816AD
:101D60008BE1F80608F033C0CD2DA7016627772751
:101D7000440F551F661F771F6A017B01A2E6B0E082
:101D800011E08D9199272D913327322F2227822B15
:101D9000932B0C01FA0110935700E89511244E5F24
:101DA0005F4F6F4F7F4FC25061F785E0F601809320
:101DB0005700E89507B600FCFDCF81E180935700FE
:101DC000E89576956795579547957A017FC080E0AD
:101DD00033DF7CC0053409F079C0F7012D2DA2E670
:101DE000B0E0EEBB8F2F99278FBB8D918DBB3196C5
:101DF000E29AE19AE199FECF215099F77F0166C0FE
:101E00008736B9F51DDF1CDFC82F1ADF863409F5C8
:101E1000C701AA27BB276C017D01CC0CDD1CEE1C81
:101E2000FF1CF60105911491802F06DF812F992761
:101E300003DF82E090E0A0E0B0E0C80ED91EEA1E09
:101E4000FB1EC25071F7F694E794D794C7947601BD
:101E500049CF853409F046CFEEBA8F2D99278FBB35
:101E6000E09A0894E11CF11C8DB3E6DEC150A1F7A5
:101E700039CF853601F596E7991641F580E090E077
:101E8000A0E0B0E023E0FC0120935700E89507B6FE
:101E900000FCFDCF805C9F4FAF4FBF4F8F3F3BE1BA
:101EA000930730E0A30730E0B30768F381E1809344
:101EB0005700E8950BC0853459F488E190E02CE098
:101EC0000FB6F894A89581BD0FBE21BD8DE02BC043
:101ED0008035E1F38C34D1F3803711F483E523C0EE
:101EE000843721F486E7A8DE80E01DC0843519F42C
:101EF000A7DE982EEBCF8B3109F4F3CE8A3A09F4A2
:101F0000F0CE863521F480E397DE81E30CC0833781
:101F100031F487E091DE83E98FDE8EE104C08B31FE
:0A1F200009F4E0CE8FE388DEDDCE89
:0400000300001C00DD
:00000001FF
